:10000E004150545832410057494445312000574918
:05001E00444532200002
:102C3B0025E0FF900297E02402F582E43401F5834E
:102C4B0022EFF0900297E004F022EFF0900296E072
:102C5B0004F0A3E004F0227B017A01790290018356
:102C6B00E0FD227C007D0A120303ED24302290024A
:052C7B009BE025E022B2
:102C8000120C29122C62122753122C6212224E7F30
:102C9000C012336FE4FF12336FE4900295F090019D
:102CA00083E0FF900295E0FEC39F501374022E1242
:102CB0002C44E0FF12336F900295E004F080DF7F38
:042CC000C002336FAC
:100C2900E4900297F0900296F0900296E090000E00
:100C3900936008122C3B122C5580EE122C3E7460E6
:100C4900122C4DE4A3F0A3F0A37408F0120F2DEFBA
:100C59006020120F2DEF122C3BEFF090029AE00466
:100C6900F07006900299E004F0122C4EA3E004F013
:100C790080DA900298E0C394065028E4900296F036
:100C8900900298E0FFC374069FFF900296E0C39F0D
:100C99005011A3122C417440122C4D900296E0047D
:100CA900F080DD7F0F7E001231F890029BEFF07F1C
:100CB900107E001231F8EF24FE602804706D122CAA
:100CC9007944E0122C3D122C4CE4900296F09002EB
:100CD90096E0900015936008122C3B122C5580EE7B
:100CE900020D2D122C7944E0122C3D122C4CE4906B
:100CF9000296F0900296E0900015936008122C3B42
:100D0900122C5580EE122C3E7462122C4DE4900286
:100D190096F0900296E090001C936008122C3B120A
:100D29002C5580EE122C3E74638009122C79446193
:100D3900122C3DEF122C4D122C3E7403122C4D1225
:100D49002C4174F0122C4D7F117E001231F8122CB7
:100D59003E122C4CE4900296F0900296E02418F58D
:100D690082E43403F583E0FF6008122C3E122C550F
:100D790080E77F127E001231F8122C3E122C4CE4CF
:100D8900900296F0900296E0240EF582E43403F581
:100D990083E0FF6008122C3E122C5580E77F137EFA
:100DA900001231F8122C3E122C4C9002FFE0FAA3EB
:100DB900E0FB7C007D64FFAE02120303EF243012D6
:100DC9002C3D122C4C7C007D0AAF03AE02120303AA
:100DD900122C6EFF122C41122C4C9002FFE0FEA344
:100DE900E0FF122C6E122C3D122C4C122C41742F48
:100DF900122C4D90030AE0FF75F064842430FE1232
:100E09002C3EEE122C4DEF75F00A8475F00A84E53C
:100E1900F02430FF122C41122C4C90030AE075F09B
:100E29000A84E5F02430122C3D122C4C122C41740A
:100E39002F122C4D122C417441122C4D122C41743D
:100E49003D122C4DE4900296F0900296E0FFC39477
:100E590006501974032FF582E43403F583E0122C4C
:100E69003D122C4C900296E004F080DD900299E44A
:100E7900F0A37440F0120F39EF601B120F39122CD6
:100E89003EEFF090029AE004F07006900299E004B7
:100E9900F0122C4E80DF122C3E7420122C4D122D94
:100EA9004BE4900296F0900296E02432F582E43405
:100EB90003F583E0FF6008122C3E122C5580E712DF
:100EC9001455EF64017026122C3E7420122C4DE447
:100ED900900296F0900296E02428F582E43403F516
:100EE90083E0FF6008122C3E122C5580E7120F4553
:100EF900300826122C3E7420122C4DE4900296F0F4
:100F0900900296E024D6F582E43402F583E0FF608E
:100F190008122C3E122C5580E7900297E09001832D
:030F2900F07F0155
:100F2C0022900299E0FEA3E0FF1231F82290029980
:090F3C00E0FEA3E0FF1231F822EF
:102BA800E0FAA3E0FBFFAE02120303EF2430FF902C
:102BB800029FE02428F582E43403F583EFF09002C5
:102BC8009FE004F0227C00AF03AE021203037C00F6
:102BD8007D0A120303ED22E02428F582E43403F58C
:0D2BE8008322E0FAA3E0FB7C007D0AFF22BF
:10145500122FD8EF7002FF227FCC1200267F441294
:10146500002630A0FD122FD8EF7002FF227FCC128C
:1014750000267FBE120026123076900330E4F0A3DA
:10148500EFF012307690032EE4F0A3EFF0E4900233
:101495009FF090029FE0FFC39406500C74282F1212
:1014A5002BE2E4122BC580EA90032EA3E0FF30E780
:1014B5001DD20BFE900331E02400FF900330E03E87
:1014C500FEEFF4FFEEF4FEEF2401FDE48012C20B03
:1014D50090032FE0FE900331E02400FD900330E0FF
:1014E5003EFCE41201F1E4FBFA7920783F12004654
:1014F50012022A9002A0EEF0A3EFF0E490029FF012
:10150500300B08122BDF742D122BC5C39002A1E0FE
:1015150094649002A0E09400500C122BEAAE0212E3
:101525000303EF02158EC39002A1E094E89002A098
:10153500E09403502C7C007D64122BA87D0A122BAD
:10154500CD2430FF122BBA122BDF742E122BC5A31C
:10155500E0FEA3E0FF122BD62430FF90029F021578
:10156500A8C39002A1E094109002A0E094275041F6
:101575007C037DE8122BA87D64122BCD2430FF124D
:101585002BBAA3122BEA122BD1122BB4122BDF7418
:101595002E122BC57C007D0AAF03AE02120303EDAC
:1015A5002430FF122BBA122BDF7443122BC57F0197
:0315B500227F0092
:0115B8002210
:0731AD001231B4D2A07F0132
:1031B400AE071FEE600D00000000000000000000DC
:0431C4000080ED2278
:102FD800D2D7C2A07FF01231B47FF01231B4D2A0A0
:102FE8007F3C1231B4A2A07FF01231B47FB4123109
:0A2FF800B420D7037F01227F0022DE
:10307600E4FDFCEDC313FDC2A07F011231AD30A00B
:1030860004ED4480FD7F3C1231B40CECB408E4AF8F
:013096000534
:013097002216
:02002600AD0724
:10002800E4FCC2A07F011231B4EDC313FD92A07F9E
:090038003C1231AD0CECB408E9F6
:01004100229C
:101F2400EF2430F09002CBE0FCA3E0FDA3E0FEA39D
:101F3400E022FFEE3395E0FDFCE0F8A3E0F9A3E036
:101F4400FAA3E022FFE4FAF9F8122CC4AC00AD01C4
:101F5400AE02AF039002CB0204E4F00B74D62BF56F
:101F640082E43402F58322A804A905AA06AB07E09B
:101F7400FEA3E0FFEE3395E0FDFC222FFFEA3EFED8
:101F8400E93DFDE83CFC2212036E78101204BD907A
:101F940002AB1204E49002AB221204BD9002A70229
:101FA40004E4EF2402FFE43EFEE43DFDE43C22F8B9
:101FB400E0FEA3E0FFE4FCFD12036E780F22FF12A3
:0F1FC4002CC4EF243022FB12036E780C0204BDF4
:1021B500121F587BA07A8679017800121F28FF121A
:1021C5002CC49002E5121F24FF7BA07A8679017842
:1021D50000121F4DE47B107A27F9F8121F28FF1211
:1021E5002CC49002D0121F24FFE47B107A27121F03
:1021F5004BE47BE87A03F9F8121F28121FC29002FC
:10220500EF121F27FFE47BE87A03121F4BE47B6480
:10221500FAF9F8121F28121FC29002F0121F277B2D
:1022250064121F48E47B0AFAF9F8121F28121FC22C
:102235009002CF121F277B0A121F489002CBA3A33F
:09224500A3E024309002D1F02244
:0D32AC00E4FF9002CBE004F00FEFB46EF5EC
:0132B90022F2
:0E32BA00E4F5D875F9DCF5E9D2DE30DFFD224F
:0F326100D2A4D2A31232ACC2A41232ACC2A322A6
:0C333500C2A4D2A31232ACD2A40232AC6B
:0E32C800A20B92A4D2A31232ACC2A30232AC6B
:10320F00D2A31232ACA2A430A404C2088002D20806
:06321F00C2A31232AC2232
:02315900AE07BF
:10315B00E4FDEE25E0FE92A4D2A31232ACC2A31280
:0A316B0032AC0DEDB408EB02320F98
:1030BA00E4FED2A4FDEE25E0FED2A31232ACA2A415
:1030CA00E4334EFEC2A31232AC0DEDB408E7AF06EC
:0130DA0022D3
:022E0000AC071D
:102E02001232617FEE123159AF041231591232611E
:102E12007FEF1231591230BAAC07C20B1232C8120C
:102E220030BAAD07D20B1232C81233351232BAAFF2
:052E320004EFFEEDFFBE
:012E37002278
:1030DB001232617FEE1231597FF41231597F2E1269
:1030EB0031591233351232BA7FF6122E00121F7875
:0130FB0022B2
:103002007F007E007D007C001232617FEE1231591A
:103012007FF41231597F341231591233351232BAD8
:083022007FF6122E00E4FDFC14
:01302A002283
:1022E6007FAA122E009002F3EEF0A3EFF07FAC125D
:1022F6002E009002F5EEF0A3EFF07FAE122E0090C6
:1023060002F7EEF0A3EFF07FB0122E009002F9EE86
:10231600F0A3EFF07FB2122E009002FBEEF0A3EFD7
:10232600F07FB4122E009002FDEEF0A3EFF07FB620
:10233600122E009002D2EEF0A3EFF07FB8122E001C
:102346009002D4EEF0A3EFF07FBA122E009002E6D0
:10235600EEF0A3EFF07FBC122E009002E8EEF0A3A1
:10236600EFF07FBE122E009002EAEEF0A3EFF0220D
:100F45001230DB90029F1204E41230029002A312C9
:100F550004E49002FDE0FEA3E0FBAA0690029F12C6
:100F65001F2BC39BFBEE9AFAED9400F9EC940090CD
:100F750002FB121FB3121F9D9002E8121F73780B1C
:100F85001204D1C004C005C006C007A3E0FEA3E05B
:100F95009002A7121F362FFBEA3EFAE93DF9E83C1D
:100FA500F8D007D006D005D004122CC4121F931216
:100FB5001F2BFF9002A7121F3D121F7F9002AF1239
:100FC50004E49002AF121F2B2408121FA9FC780419
:100FD5001204BD1221B59002F0E09002E0F09002FB
:100FE500CFE09002E4F09002D1E09002ECF09002A4
:100FF500AF121F2B2460FFEE34F0FEED34FFFDEC45
:1010050034FFFCA31204E49002B3121F2BFFA804C3
:10101500A905AA06121FCA9002D4121F6B12036EED
:10102500780B121F9D9002F5E0FEA3E09002B3122B
:101035001F36FB12036E780B121F90121F2BFF90A9
:1010450002A7121F3D121F7F9002B71204E49002FF
:10105500F3121F73E47B04FAF9F812036E9002B7DA
:10106500121F3D121F7F121FA6FCE47B04FAF9F83C
:10107500122CC49002BB1204E49002F7121F739065
:1010850002B3121F3DFB12036E780D121F9D9002D5
:10109500B3121F2BFF9002B3121F3D121FCA9002FD
:1010A500D2121F6B121F8B121F2BFF9002A7121F4C
:1010B5003D121F7F121FA6FC78021204BD9002B7D5
:1010C5001204E49002B7121F2B2400FFEE348012A5
:1010D5001FACAB07AA06A9059002F9121FB31204AB
:1010E500AA9002C31204E49002A3121F2BFFC004AE
:1010F500C005C006C0079002BB121F2BFBAA06A99C
:1011050005A804D007D006D005D004C3EF9BFFEE99
:101115009AFEED99FDEC98FCE47B507AC3F9F81240
:10112500036E9002C71204E4E4FFFEFD7C8090028A
:10113500C7121F3DFBC3120499501EE47F02FEFD3A
:10114500FC9002C7E0F8A3A3A3E012036E9002C3CC
:10115500121F3DFB1203F980189002C3121F3DFBBD
:10116500A3121F2BFF1203F9E47B02FAF9F812030D
:101175006E9002BF1204E49002BF121F2BFF780885
:101185001204BDC004C005C006C0079002BF121FEF
:101195002BFF78081204BDD003D002D001D0001275
:1011A500036E121FA0E47FDE7E0BFDFC9002A712EA
:1011B5001F3DFB12036E7810121F9D7F437EE37D5A
:1011C500FF7CFF9002BF121F3DFB121F8B121F2BCE
:1011D500FF9002A7121F3D121F7FEF24CFFFEE34B1
:1011E5000E121FACFC78041204BD9002BF121F3D05
:1011F500121F7F1221B59002E5E0FF9002EEF090FC
:1012050002D0E0FE9002F2F09002EFE0FD9002E1E4
:10121500F09002F0E0FC9002EDF09002CFE0F99042
:1012250002F1F0E4FB24D6121F63EF121F5EEE12EB
:101235001F5EED121F5EEC121F5E742E121F5EE91B
:0F124500121F5E7470F074D62407121F63E4F05A
:011254002277
:10259B001203F9EB2430FF9002A3E02432F582E41E
:1025AB003403F583EFF09002A3E004F0E02432F55E
:1025BB0082E43403F583227F07122E38E4FCFD12EC
:1025CB0001ECE4FBFA79407840120046E4FBFA791F
:1025DB0080784412014FE4FBFA227B0AFAF9F89057
:1025EB00029FE0FCA3E0FDA3E0FEA3E0FF227948FD
:0F25FB00784312004602022A900293E0940122D4
:0D330E00439180439280439D8075BCA022B6
:102E3800E4F5BDF5BEE5BC54E044084FF5BC000020
:102E480000007DFAE5BC30E41753BCEFAFBDEF7569
:102E5800F004A4FFACBEEC7A002FFFEA35F0FE22A6
:062E6800DDE27E037FFFA6
:012E6E002241
:102D4B001225C279A078411225FD90029F1204E44E
:102D5B00E49002A3F01225E51203F9E47B0AFAF9D9
:102D6B00F812259B742EF09002A3E004F0E41225D8
:102D7B00E512259B74561225B0E4F09002A3E004F3
:012D8B00F057
:012D8C002224
:102887001225C21225F9900293EEF0A3EFF0C3943C
:102897009AEE940140047F068042C3900294E0942C
:1028A7007C12260340047F058032C3900294E09493
:1028B7005E12260340047F048022C3900294E094B2
:1028C7004012260340047F038012C3900294E094D1
:0F28D7003112260340047F0280027F011230522B
:0128E60022CF
:10267900E490029BF0A3F0A3F07F07122E38E4FC4C
:10268900FD9002971204E49002971225EDE41225B9
:10269900CA1225F99002931204E4900293A3122519
:1026A900F290029CE02FF090029BE03EF090029D98
:1026B900E004F0E0C3940A40C090029BE0FEA3E06E
:1026C900FF7C007D0A12030390029BEEF0A3EFF05A
:0D26D900C39431EE940150037F01227F0075
:0126E60022D1
:10305200900295EFF0900295E0FF14F0EF6014C239
:10306200907F037E0012311DD2907F037E001231C9
:043072001D80E222B9
:10311D00EF4E6019EF1FAC0670011E4C600FE4F509
:0E312D00D875F94CF5E9D2DE20DFE980FB22EF
:0D331B00D2C2D280D290D282D283D281223F
:103175001226E712336512313B1228E71229FF1296
:0C3185002118122679BF01EBC20980E777
:10313B0020961A7F017E0012311D209610B284302A
:0E314B0096FD7F017E0012311D3096F3222288
:102F57002096277F017E0012311D20961D7F0112CA
:102F670015B9C2C2C290C282C2813096FD7F017E6E
:0B2F77000012311D3096F375C72022B8
:030003000229A52A
:1029A500C0E0C0F0C083C082C0D075D000C000C0F8
:1029B50001C002C003C004C005C006C00720B21F85
:1029C5007F017E0012311D20B215B20930B2FD7FA4
:1029D500017E0012311D30B2F330090375C720D0D6
:1029E50007D006D005D004D003D002D001D000D046
:0A29F500D0D082D083D0F0D0E032C1
:0A3365002009061232D675870222F5
:0E32D600C294C284C2C0D2B6D2B712331B2239
:1026E7001232D6D209D2C012338075BBFFE4F591FE
:1026F700759220F5B375B40143B70243B80243B7E7
:1027070010C2C2C280C290C282C283C2817F0AFE47
:1027170012311D12331B1231E0122F5712330E12D2
:1027270032701233871222E61214551214551230E2
:102737002BC28CE490033CF0C28CC28D758C4CF597
:0C2747008AD28CD2A8D2A9D2AF02288777
:03000B00022AAF17
:102AAF00C0E0C0F0C083C082C0D075D000C000C0ED
:102ABF0001C002C003C004C005C006C007C28CC25B
:102ACF008D758C4C758A00D28C90033CE004F0E03D
:102ADF00D394144005E4F0122496D007D006D00505
:102AEF00D004D003D002D001D000D0D0D082D08378
:052AFF00D0F0D0E03230
:1016F100504F5745523A200020202054454D503A32
:101701002000202D2D2D2D2D200020202050726510
:1017110073737572653A2000200D0A0D0A00415459
:101721002B48454C503D310D0A0041542B44454D49
:101731004F3D310D0A0041542B43414C4C3D000DAE
:101741000A0041542B535349443D0041542B444911
:1017510047493D0041542B54494D453D0041542BCF
:10176100424541434F4E3D000D0A0D0A002A2A2AE7
:101771002041505253203531547261636B205832ED
:101781004128424C41434B424F5829203230313499
:10179100313031322042483454445620202A2A2AFA
:1017A100200D0A004E4F43414C4C00333133342E4F
:1017B10035354E000031323032302E36364500415B
:1017C100505253203531547261636B20583241209D
:1017D10021000000000000000000000000312C3456
:1017E10033382E353030302C3433382E35303030DC
:1017F1002C302C332C300000000000312C313434DB
:101801002E363430302C3134342E363430302C30C6
:091811002C332C302C30000000B7
:1028260090029CE0FEA3E0FFE4FD123191E004F08B
:102836002290029BA3E02400F582E43400F5832273
:1028460090029BE0FEA3E0FF2290029CE004F022AF
:1028560090029CE0FEA3E0FF2290029BE004F0229F
:1028660075C65A75C6A52290029CE4F0A322ECF523
:10287600C3AF058FC422F0A3EFF0C3940AEE940011
:01288600222F
:10089600E490029DF0A3F090029BF0A3F090029DDD
:1008A600E0FEA3E0FF1231F8122837EFF090029E27
:1008B600E004F0700690029DE004F090029CE004D3
:1008C600F0700312285FC390029BE0940140CE7B38
:1008D600FF7A17796E122EFF122D4B7BFF7A16794F
:1008E600F1122EFF7B017A037932122EFF7BFF7AFB
:1008F6001679F9122EFF121455BF01087B017A03EF
:10090600792880067BFF7A177903122EFF7BFF7A00
:1009160017790B122EFF120F453008087B017A0259
:1009260079D680067BFF7A177903122EFF7BFF7A32
:10093600177919122EFF7BFF7A17791F122EFF7B6C
:10094600FF7A17792B122EFF7BFF7A177937122E33
:10095600FF90029BE4F0A37408F0122837E0FF60D2
:100966000A120BF170F412285F80EF120BD47A177B
:100976007943122EFF90000FE0FF7E0090029BEE5F
:1009860012287C1228467C007D0A5002800A120B2F
:10099600A61228467C007D0A120C07120BD47A1781
:1009A600794C122EFF900005120BC7900006120B11
:1009B600C7900007120C12900004E02430FF123397
:1009C6006F120BFB7A177955122EFF900000E0FE8E
:1009D600A3E07C002400FFEC3EFE90029B12287CE4
:1009E600500B90029BA3E02430FF12336F1228466F
:1009F600D39409EE940040047D0180027D00C3EF8C
:100A06009464EE940050047F0180027F00EF5D60E5
:100A160003120B72122846D39463EE940040047DB1
:100A26000180027D00C3EF94E8EE940350047F0139
:100A360080027F00EF5D600D1228467C007D641207
:100A46000BA6120B72122846D394E7EE94034004C9
:100A56007D0180027D00C3EF9410EE942750047F41
:100A66000180027F00EF5D6006120B12120BB812B6
:100A76002846D3940FEE942740147C277D1012034A
:100A860003120BB8120B127C007D0A120C07120B14
:100A9600FB7A17795E122EFF900010120C1290004E
:100AA60011120BE07420F0122837E0FF600A120BD7
:100AB600F170F412285F80EF7F2C12336F900012D2
:100AC600120BE07430F0122837E0FF600A120C1F98
:100AD60070F412285F80EF7F2C12336F900013E0C2
:100AE600FF12336F7F2C12336F90029BE4F0A374D6
:100AF60040F0122837E0FF600A120C1F70F412282B
:0C0B06005F80EF7BFF7A177969022EFFF9
:100B120090029BE0FEA3E0FF7C037DE81203037CCE
:100B2200007D0A120303ED2430FF12336F90029B03
:100B3200E0FEA3E0FF7C007D641203037C007D0ADB
:100B4200120303ED2430FF12336F90029BE0FEA3E9
:100B5200E0FF7C007D0A1203037C007D0A1203037E
:100B6200ED2430FF12336F90029BE0FEA3E0FF22E0
:100B720090029BE0FEA3E0FF7C007D0A1203037C4F
:100B8200007D0A120303ED2430FF12336F90029BA3
:100B9200E0FEA3E0FF7C007D0A120303ED2430FF98
:100BA20012336F221203037C007D0A120303ED2429
:100BB20030FF12336F227C007D0A120303ED2430D2
:100BC200FF12336F22E02430FF12336F7F2C123377
:100BD2006F227BFF7A177940122EFF7BFF22E0FF04
:100BE20012336F7F2C12336F90029BE4F0A3221218
:100BF200336F90029CE004F0227BFF7A1779401257
:100C02002EFF7BFF22120303ED2430FF12336F22EB
:100C1200E02430FF12336F7F2C12336F2212336FB6
:070C220090029CE004F022A7
:1031C80090029EEFF07F007E0212323B90029EE05A
:0831D800FD7F007E020231912F
:102B5700E4FFFE12323BE490029DF0A3F090029B4B
:102B6700F0A3F090029BE0FCA3E0FDC3EC940150BE
:102B77002FA3E0FEA3E0FF74002D12283EE0FD1214
:102B8700319190029EE004F0700690029DE004F0FF
:102B970090029CE004F070CB90029BE004F080C3AD
:012BA700220B
:1031E0007F1F7E001231F8EF64997F01600912158C
:0831F000B975C7207F002222FF
:0E32E400E4F5C7F5C5F5C675C3FF75C4FF2236
:0431F800AD07AC066D
:1031FC0075C78275C50112287412286600AFC212F9
:02320C0032E4AA
:01320E00229D
:10323B00AD07AC0612287475C78275C503122866D4
:03324B000232E468
:102ED200AD07AC0675C78275C5021228741202AB23
:102EE200F5C2122866000DBD00010C740129F9E437
:0D2EF2003AFA9002A3E014F070E00232E41E
:10319100AB07AA0675C78275C502EAF5C3AF038FEF
:0C31A100C4AF058FC2122866000232E4A1
:0515B90090029BEFF021
:1015BE00E4FFFE12323B7BFF7A1779A59002A374EB
:1015CE0007F07F08122ED27D097F0F1231917D0117
:1015DE007F041231911D7F051231917F06123191D8
:1015EE000D7F071231910DE4FF1231917D587F016D
:1015FE001231917D017F101231917D217F111231B7
:10160E00917D2F7F121231917D3E7F1312319112F7
:10161E00286D7420F0E4FCEC9017AC93FD600E1274
:10162E002856122830700312284F0C80EA122826F2
:10163E00700312284F12286D7430F0E4FCEC9017F2
:10164E00B693FD600E122856122830700312284FE2
:10165E000C80EA122826700312284F12286D74404F
:10166E00F0E4FCEC9017C093FD600E122856122881
:10167E0030700312284F0C80EA12282670031228AD
:10168E004F90029BE07028A3F0A37480F0E4FCEC72
:10169E009017DE93FD600E1228561228307003123A
:1016AE00284F0C80EA122826700312284F8026122B
:1016BE00286D7480F0E4FCEC9017FC93FD600E1224
:1016CE002856122830700312284F0C80EA12282652
:1016DE00700312284F7D997F1F7E00123191E4FF17
:0316EE000231C8FE
:101DC4000D0A2020B2BBC8CFCAB6C4E3CAE4C8EB2C
:101DD400B5C4D6B8C1EEA3ACBFC9C4DCC3BBBCD3C5
:101DE400BBBBD0D0C5B6A3A120A3BAA3A920200D04
:101DF4000A0D0A0041542B48454C503D31004154D2
:101E04002B44454D4F3D310041542B54494D453DE4
:101E14000041542B43414C4C3D0041542B535349F6
:101E2400443D0041542B424541434F4E3D004154F3
:101E34002B444947493D000D0A202D3E20C9E8D6D0
:101E4400C3B3C9B9A620202120200D0A000D0A2001
:101E54002D3E20D6B8C1EEB4EDCEF3A3A1BFC9C4C4
:101E6400DCC8B1C9D9BBD8B3B5A3A120200D0A00E1
:101D0500900294E02400F582E43400F583E4F09039
:101D15000293E004F0E02407F582E43402F583E061
:101D250022900210E024D0FFE434FFFE7C00120272
:101D3500F1AA06AB0790020FE024D0FFE434FFFEC2
:101D450022900294E02400F582E43400F5832274A5
:101D550008900293F0E4900297F0A3F022EFF09040
:101D65000293E004F022900298E004F0229002979A
:101D7500E004F0227D0A1202F1EF2BFFEE3AFE227B
:101D8500900287E0FF2406F582E43402F583E02221
:101D95001202F1EF2BFBEE3AFA22900294F0900238
:101DA50093227B017A017902900183E0FD22900262
:0F1DB50097E0FEA3E0FFEE2290020FE024D02281
:030023000227BFF2
:0D27BF00C0E0C083C082C0D075D000C0074C
:1027CC00309906C299D2078046309843300604C22D
:1027DC0098803C7F80900207E4F0A3DFFC7F0075BB
:1027EC00D80075F94C75E900D2DE20980C30DFFA70
:1027FC00900287EFF0D2068016C29874072FF582EC
:0F280C00E43402F583E599F00FEFD3947F40D0C9
:0B281B00D007D0D0D082D083D0E032B4
:102118002006030221B4900207E064C0704EA3E0D9
:10212800704A121D8564C07043EFD39411403DE49A
:10213800900183F07F02900287E014FEEFC39E5067
:102148001C74072F121D1DFE74002FF582E4340144
:10215800F583EEF0900183E004F00F80D9121DA7FB
:10216800122753121DA712224EC20622121D85B431
:102178000A047E0180027E0074052FF582E4340291
:10218800F583E0B40D047F0180027F00EF5E6008F4
:10219800E4F5AF1204F0800FE4F5AF1208967BFF68
:0C21A8007A1D79C4122EFFC206123328E3
:0121B4002208
:1004F000E4900299F0A3F0121D5B900299E0FEA334
:10050000E0FF1231F8900297A3121D49EFF090021C
:100510009AE004F07006900299E004F0121D6B70EE
:1005200003121D72C3900297E0940140CD7BFF7AC5
:100530001D79F81230FCBF01030208967BFF7A1E7A
:1005400079021230FCBF010BE4FF1215B9123341DE
:1005500075C7207A1E790C120873600302063412E4
:100560001D54900293121D1A640D600D121D641229
:100570001D6B70EE121D7280E9121DB3600302063E
:100580001BEF24FE602114602A14603714604E248F
:1005900004600302061B121DBDFEE434FF900295A9
:1005A000F0A3CEF0020622121D3A7C007D0A120250
:1005B000F180277D0A121D267D64121D7B90021199
:1005C0000206067D64121D267C037DE8121D9590AF
:1005D0000211121D3D7C00121D79A380299002108A
:1005E000121D3D7C037DE8121D337C277D10121DFA
:1005F00095900211121D3D7C007D64121D95A31281
:100600001D3D121D79A3E024D0FDEC34FFCD2FFF5A
:10061000ED3E900295F0A3EFF08007E4900295F094
:10062000A3F0900295E0FCA3E0FDEC900000F0A3A5
:10063000ED12088E7A1E79151208737074121D540B
:10064000900293121D1A640D600D121D64121D6B31
:1006500070EE121D7280E9D3900298E09406900229
:1006600097E09400400312334D900297E07002A38C
:10067000E0700312334D7408121D9FF0900298E051
:100680002408FF900297E03400FE900293E0FDC33F
:100690009FE49E501674072D121D1DFF121D46EF7C
:1006A000F0900294E004121D6380D1121D461208DE
:1006B0007C7A1E791E120885704B121D549002938D
:1006C000121D1A640D600D121D64121D6B70EE1266
:1006D0001D7280E9121DB37020EF24FE60080470C3
:1006E00018121DBD800D121DBD75F00AA4FFA3E0F8
:1006F00024D02F90000FF0800690000F740AF012A3
:100700002B571233417A1E7927120885600302079E
:10071000F0740A121D56900293121D1AFF640D60A8
:1007200011EFB42C08121D6B7003121D72121D64A0
:1007300080E4900297E07004A3E06406600302087E
:1007400029900293740A121D1924D0900010121DD2
:1007500013642C600312334D121D14900011121DEE
:1007600013642C600312334D7420121D9F8012906D
:100770000293121D1AFF642C600C121D46121D629A
:10078000A3E004F080E9121D05900012121D13640D
:100790002C600312334D9002947430F090029380D9
:1007A00012900293121D1AFF642C600C121D461247
:1007B0001D62A3E004F080E9121D05900013121DD4
:1007C00013642C600312334D9002947440F0900235
:1007D000938012900293121D1AFF640D600C121D7B
:1007E00046121D62A3E004F080E9121D4612087C47
:1007F0007BFF7A1E79321230FCEF64017074121D97
:1008000054900293121D1AFF640D6011EFB42C086E
:10081000121D6B7003121D72121D6480E49002970A
:10082000E07004A3E06403600302334D900293740C
:1008300008121D1924D0900005121D13642C6003AA
:1008400012334D121D1424D0900006121D13642C77
:10085000600312334D121D1424D0900007121D1393
:10086000642C600312334D121D1424D09000041226
:02087000088EF0
:10087200227BFF1230FCEF640122E4F0122B5712AC
:100882003341227BFF1230FCEF640122F0122B571E
:0408920012334122BA
:0C3341001208967BFF7A1E793B022EFFDB
:0C334D001208967BFF7A1E7951022EFFB9
:1030FC00E4FF1202ABFE601674072F121D1D6E60EA
:10310C00037F00220F740129F9E43AFA80E47F016D
:01311C002290
:0F327000759850759CFD758E1175891102322568
:10322500C2ACC206E4900287F07F80900207E4F00A
:05323500A3DFFCD2AC98
:01323A002271
:102EFF0090029FEBF0A3EAF0A3E9F090029FE0FBB2
:102F0F00A3E0FAA3E0F91202ABFF600F12336F9048
:0C2F1F0002A0E475F00112035880E022CB
:0A336F00C2078F993007FDC2072244
:101939000F90028BE0FBA3E0FAA3E0F98F82758395
:10194900000202C4FD74182EF582E43403F583ED18
:10195900F00E0F2290028BE0FBA3E0FAA3E0F9223C
:1019690090028CE0900304F090028DE0900305F062
:1019790090028EE0900306F090028FE0900307F04A
:101989009002902290028DE0900304F090028EE084
:10199900900305F090028FE0900306F0900290E02A
:1019A900900307F090029122FD740E2EF582E43423
:1019B900032290028CE0900305F090028DE09003E1
:1019C90006F090028EE0900307F090028F229002B9
:1019D9008BE0248CF582E43402F583EEF090028BDF
:1019E900E004F00F22EBF0A3EAF0A3E9F0E422907F
:1019F900028CE0900306F090028DE0900307F090CE
:101A0900028E22F09002FFE0FFA3E0900322CFF0C4
:101A1900A3EFF07F012290028EE024D022748E2D54
:101A2900F582E43402F583EFF00C0D22C294C20072
:101A3900D28022FFE434FFFE7C007D0A0202F1908D
:0B1A4900028CE0900307F090028D2259
:102E6F0020932E7F017E0012311D20932490032585
:102E7F00E004F0E0D394044002E4F0900325E0FF77
:102E8F001231C83093FD7F017E0012311D3093F354
:022E9F002222ED
:1029FF00122E6F900325E024FE60151460331460CF
:102A0F0033240370339003247401F0D294022F2BDC
:102A1F00900324E064026003122EA1900324740239
:102A2F00F0D294300222C20230001D122C80C2005C
:102A3F0022022A58121A3522E4900324F02094051A
:092A4F00123328D294122F8222C6
:102EA100E4FFFE1231F8EF7F00FEC006C0070F7E7F
:102EB100001231F8EFFDD0E02DFFD0E03400FE909C
:102EC1000326F0A3EFF0900301EEF0A3EFF0C202AE
:012ED10022DE
:102A5800900324E0640360097403F0121A35122EFF
:102A6800A1300242C202123328D294E4900293F0B9
:102A7800A3F02000287F147E0012311D900294E0FC
:102A880004F07006900293E004F0D3900294E0946E
:102A98002C900293E0940140D9121A3522122C800E
:062AA800121A35122EA1E6
:012AAE002205
:10249600900325E024FE60121460171460252403BF
:1024A6007029D281D282B2838027B281D282D2832E
:1024B600801FD283308206C282C2818014D282D229
:1024C60081800ED281B282D2838006D282D283D21A
:1024D60081900326E0FEA3E0FF4E601F900302E01A
:1024E60024FFF0900301E034FFF0E07002A3E070F7
:1024F6000A900301EEF0A3EFF0D20290030CE00481
:10250600F0700690030BE004F0D390030CE0940403
:0F25160090030BE094004006E4F0A3F0D2012202
:102F82003091037F00227F017E0012311D309103B8
:102F92007F00223091FD7F017E0012311D3091F3BE
:0B2FA200300005122C80C2007F0122CD
:102F2B0030000D122525BF0107122C80C200801224
:102F3B0030011830000C122BF5BF0106122C80C289
:0C2F4B000022E490030BF0A3F0C201226E
:10302B00E4900322F0A3F090030DF0C20090032470
:10303B00F0122EA1E490030BF0A3F0FF7E021231ED
:07304B00F8900325EFF022CD
:031B5A009002886E
:101B5D001219EEFFFE90028812193DFD6009B42C9A
:101B6D00010E0FEEB409EE90028812193D642D702E
:101B7D00600F90028BF090028812193DFE642E606A
:101B8D00051219D780F07F069003037430F0A3DFA0
:101B9D00FC900303742DF090028BE024FE6013146F
:101BAD0060151460171460192404701A90028C02C9
:101BBD001BD6121A4880121219F8800D1219BB800B
:101BCD0008121969800312198DE0900308F0021CA8
:101BDD003EE490028BF090028812193DFE642E6057
:101BED00051219D780F07F069003037430F0A3DF40
:101BFD00FC90028BE024FE60131460161460181420
:101C0D00601A2404701B90028C021C39121A4802AF
:101C1D001C391219F880151219BB80101219698020
:101C2D000B90028CE0900303F012198DE0900308E5
:061C3D00F0E4900309F041
:011C4300227E
:032D0800900288AE
:102D0B001219EEFFFE90028812193DFD6009B42CDA
:102D1B00010E0FEEB402EE90028812193DB4411968
:102D2B007B017A017985121E747B017A01798512F8
:0F2D3B001A54C280D2007F0122B280C2007F00F2
:012D4A002266
:031E740090028B4E
:101E77001219EEFFFE12193A6009B42C010E0FEE8B
:101E8700B403F2E4FE12193AFD642E600512194EEE
:101E970080F390028B12196012194E12194512190C
:101EA7004D12194512194D12193A642C60030F800F
:101EB700F612193912194D74182EF582E43403F508
:101EC70083E4F012193A642C60030F80F60FE4FEE6
:101ED70012193AFD642E60081219B212195680F0D1
:101EE70090028B1219601219B21219561219451263
:101EF70019B11219561219451219B1121956121998
:101F07003A642C60030F80F61219391219B1F58360
:0C1F1700EDF00E1219B2F583E4F07F012A
:011F2300229B
:1025250090030AE07002FF22900322E0FEA3E0FF81
:102535009002FFE0FAA3E0FBD39FEA9E4008EB9FE1
:10254500FDEA9EFC80159002FFE0FEA3E0FFC3902C
:102555000323E09FFD900322E09EFCD3ED94B4ECB1
:102565009400401074689D900294F074019C900250
:1025750093F08008900293ECF0A3EDF0D3900294D1
:10258500E09419900293E094004008E490030D1242
:052595001A0C227F007A
:01259A00221E
:102BF50090030AE0FE7002FF2290030DE004F0EE60
:102C0500C3940A500AE0940B400280227F00229070
:102C1500030AE0C39432500D90030DE0940740027F
:102C2500800C7F002290030DE0D394054005E4124B
:062C35001A0C227F0022B0
:031A540090028B72
:101A57001219EEFCFD12195D8C821219476009B448
:101A67002C010D0CEDB407ED12195D8C821219478C
:101A7700B42C03E4804BE4FD12195D8C82121947E4
:101A8700FF642E6005121A2680EEED24FD60120415
:101A9700702C121A1F75F00AA4FFA3E024D02F8020
:101AA7002090028FE024D075F00AA4FF121A1F7548
:101AB700F064A42FFF900290E024D02F8003121A25
:101AC7001F90030AF012195D8C82121947642C606B
:101AD700030C80F10C12195D8C82121947B42C0883
:101AE700E49002FFF0A3F022E4FD12195D8C82124C
:101AF7001947FF642E6005121A2680EEED24FD605B
:101B07000C047040121A1F121A3CA3802390028FF4
:101B1700E024D0121A3CAA06AB07121A1FFFE434BE
:101B2700FFFE7D641202F1EF2BFFEE3AFE9002906A
:101B3700E024D0FDEC34FFCD2FFFED3E9002FFF007
:101B4700A3EFF022121A1FFEE434FF9002FFF0A366
:021B5700CEF0CE
:011B59002269
:0E32F200244750524D430024475047474100A7
:10309800A3F07B017A01798522900206E02485F568
:1030A80082E43401F58322E0FBA3E0FAA3E0F9020D
:0230B80002AB69
:03004300021C4458
:101C4400C0E0C0F0C083C082C0D075D000C000C066
:101C540001C002C003C004C005C006C007E59A3035
:101C6400E106539AFD021CEAE59A30E079539AFEA4
:101C74001230A1E59BF0900206E004F0900184E0AC
:101C840004F0E59B640A70531230A1E4F09002065C
:101C9400E004F0200A2190028B74FFF0A37432F068
:101CA40074F2123098122DC7EF6401702712309A23
:101CB400122D08D20A801D90028B74FFF0A3743297
:101CC400F074F9123098122DC7BF010812309A121D
:101CD4001B5AC20A900206E4F0800B900206E0D37D
:101CE400947E4002E4F0D007D006D005D004D0039F
:101CF400D002D001D000D0D0D082D083D0F0D0E0B8
:011D040032AC
:102DC700900288EBF0A3EAF0A3E9F090028B1230AF
:102DD700AFFF60229002881230AF6F60037F00223E
:102DE700900289E475F00112035890028CE475F0A3
:092DF7000112035880D57F01226E
:06338700759A5002332884
:0D332800E4F5AFC200900206F075AF01227F
:102FAD00E4F5D875F9FDF5E9D2DE22C313F04480BE
:102FBD00F0900182E004F022C2ACE4F5AFD2C2D2AF
:0B2FCD0080D29022900100E0640322FB
:1028E70020B55C122FC5121FD3900293EFF012325E
:1028F70025123328900293E064017043122FCAC255
:10290700C27FC012336FE4FF12336FE4900294F07A
:10291700900183E0FF900294E0FEC39F501774027A
:102927002EF582E43401F583E0FF12336F900294B1
:0F293700E004F080DB7FC012336FD2C212324E49
:01294600226E
:0E224E00900297EBF0A3EAF0A3E9F0A3EDF005
:10225C00122FC5C290C2B6D2B7D295D2B39001821A
:10226C00F090029BF01222DAE0C3944C40F7E49019
:10227C00029BF090029AE0FFA3E0C39F50249002CF
:10228C0097E0FBA3E0FAA3E0F91202ABFF12294797
:10229C00900298E475F00112035890029BE004F050
:1022AC0080D190033BE0FF12294790033AE0FF12E4
:1022BC002947E490029BF01222DAE0C3940A40F71B
:0E22CC00D2B6C2B7C295D29012322502332884
:0C22DA007F7E12294790029BE004F02256
:101FD300122079122FD160037F0022900101E0B417
:101FE3007E0B12260A122FD160F17F0022E49002A9
:101FF30095F0900101E0FF647E602C900295E0244F
:1020030002F582E43401F583EFF0900295E004F0E9
:1020130012260A900295E0D3947840037F0022129F
:102023002FD160CE7F00227B017A01790290029545
:10203300E024FEFD122753900295E0FE2400F58272
:10204300E43401F583E0FF90033BE06F60037F001E
:102053002274012EF582E43401F583E0FF90033A04
:10206300E06F60037F0022900295E024FEF0E09091
:052073000183F07F0174
:012078002245
:10207900E4900100F0123379123379E4900101F010
:1020890030B40A30B5FA9001007401F02220B40A84
:1020990030B5FA9001007402F022A2B49204E490DF
:1020A9000182F0900296F012328E900101E0C31382
:1020B900F0900182E0B40616900296E004F0E0B4D4
:1020C900030C9001007403F0E4900182F022E49083
:1020D9000182F0C2052005CF122FAD20DF1C30B5DB
:1020E900079001007404F022A2B4300401B350EB4C
:1020F900A2B49204D205D2DF80E12005D890010173
:0E210900E0122FB8E0B407CD9001007405F08D
:0121170022A5
:10260A00E4900296F0900296E0C394085060122F6C
:10261A00AD20DF2030B5079001007404F022A2B487
:10262A00300401B3500AA2B49204D205D2DF80E189
:10263A00C20580DD200515900101E0FF122FB8E0E8
:10264A00B407079001007405F022801A12328E90A6
:10265A000182E0B40504E4F080AB900101E0C31309
:0E266A00F0E4900182F0900296E004F0809778
:01267800223F
:0529470090029CEFF07E
:10294C00BF7E04D2038002C203E490029DF0900289
:10295C009CE054017004B2B38023122FBE200304F8
:10296C007F0180027F00900182E0B405047E01802B
:10297C00027E00EE5F600A12327FB2B3E4900182F5
:10298C00F090029CE0FFC313F012327F90029DE0A6
:08299C0004F0E0C3940840B60A
:0129A4002210
:0F327F00E4F5D875F9FD75E908D2DE30DFFD22E0
:07337900122FAD30DFFD2231
:0F328E00E4F5D875F9FE75E980D2DE30DFFD2258
:07338000C295D2B6C2B722CC
:10125500000011892312329B462457AD653674BFB1
:101265008C489DC1AF5ABED3CA6CDBE5E97EF8F761
:10127500108101083393221A56A5472C75B7643E91
:101285009CC98D40BFDBAE52DAEDCB64F9FFE87641
:101295002102308B02101399672676AF443455BD71
:1012A500AD4ABCC38E589FD1EB6EFAE7C87CD9F521
:1012B5003183200A1291031877A7662E54B5453C51
:1012C500BDCBAC429ED98F50FBEFEA66D8FDC97401
:1012D5004204538D6116709F042015A9273236BB31
:1012E500CE4CDFC5ED5EFCD7886899E1AB7ABAF3E1
:1012F5005285430C7197601E14A1052837B3263A11
:10130500DECDCF44FDDFEC5698E98960BBFBAA72C0
:101315006306728F4014519D252234AB063017B9F0
:10132500EF4EFEC7CC5CDDD5A96AB8E38A789BF1A0
:101335007387620E5095411C35A3242A16B10738D0
:10134500FFCFEE46DCDDCD54B9EBA8629AF98B7080
:1013550084089581A71AB693C22CD3A5E13EF0B7B0
:10136500084019C92B523ADB4E645FED6D767CFF60
:1013750094898500B79BA612D2ADC324F1BFE03690
:1013850018C109483BD32A5A5EE54F6C7DF76C7E40
:10139500A50AB48386189791E32EF2A7C03CD1B570
:1013A500294238CB0A501BD96F667EEF4C745DFD20
:1013B500B58BA40296998710F3AFE226D0BDC13450
:1013C50039C3284A1AD10B587FE76E6E5CF54D7C00
:1013D500C60CD785E51EF497802891A1A33AB2B330
:1013E5004A445BCD695678DF0C601DE92F723EFBE0
:1013F500D68DC704F59FE41690A98120B3BBA23210
:101405005AC54B4C79D7685E1CE10D683FF32E7ABF
:10141500E70EF687C41CD595A12AB0A3823893B1EF
:101425006B467ACF485459DD2D623CEB0E701FF99F
:10143500F78FE606D49DC514B1ABA02292B98330CF
:101445007BC76A4E58D5495C3DE32C6A1EF10F787F
:05275300900297EDF07B
:1027580074FFA3F0A3F0900297E0D39400403F12D7
:1027680002ABFF900298A3E06F25E0FFE433FE740C
:10277800552FF58274123EF583E493FC740193FDA2
:10278800900298E0FFECFEED6FFFEEF0A3EFF09003
:102798000297E014F0740129F9E43AFA80B890023B
:1027A80098E0FEA3E0F4FFEEF4FCEF90033BF0AEFC
:0627B80004EE90033AF06C
:0127BE0022F8
:0E3300005749444531200057494445322000CA
:102B04001FEF25E0FF74022EF582E43401F583ED16
:102B140054E1F074022EF582E43401F58322749DAD
:102B24002FF582E43402F58322F0900298E004F059
:102B340022EE75F007A414F0AF067BFF227B017A26
:102B4400017902900183E0FD2290029BE4F0A374DA
:032B540008F02264
:10324E0090010FE020E00B122376EF640160031271
:03325E0024062221
:102376009002957403F07F057E001231F8EF640138
:10238600707B900295E0FED3940840037F00229074
:102396000296122B357A337900122D8DEF64017077
:1023A60043900296E0FE2402122B1AE0FD541EC34F
:1023B60013FF7002FF22122B04E04FF0EF700D9016
:1023C6000296E02402122B1AE04480F07F077E007A
:1023D6001231F8BF0108900295E0FF12181A123266
:1023E6009D7F0122900296E02402122B1AE030E033
:0F23F600037F0022900295E004F00223887F000D
:0124050022B4
:102406009002957403F07F067E001231F8EF6401A6
:10241600707B900295E0FED3940840037F002290E3
:102426000296122B357A337907122D8DEF640170DF
:1024360043900296E0FE2402122B1AE0FD541EC3BE
:1024460013FF7002FF22122B04E04FF0EF700D9085
:102456000296E02402122B1AE04480F07F077E00E9
:102466001231F8BF0108900295E0FF12181A1232D5
:102476009D7F0122900296E02402122B1AE030E0A2
:0F248600037F0022900295E004F00224187F00EB
:012495002224
:102D8D00EF1475F007A4900297F01202AB6028259E
:102D9D00E0FFE433FE900297E02402122B1AE06F5D
:102DAD007001EE60037F0022740129F9E43AFA9074
:092DBD000297E004F080D37F01CD
:012DC60022EA
:05181A00900297EFF0C1
:10181F00900183E0D394784003021938122B4DFFC7
:10182F007E001231F8EF7003021938122B4DE4903D
:10183F000298F0900298E0FFC39406500A122B22F0
:10184F007440122B2D80ECE4900298F090029BE0F4
:10185F00FEA3E0FF1231F890029AEFF06029900298
:10186F009AE025E0FF900298E0249D122B25EFF0DF
:10187F0090029CE004F0700690029BE004F0122BA3
:10188F002EE0C3940640C57F0F7E001231F8EF257E
:10189F00E044E09002A3F0900299E004F0900183FD
:1018AF00E0FF90029AF0900297E075F007A424F8F9
:1018BF00FEC3EF9E900299F0E4900298F090029987
:1018CF00E0FF900298E0C39F502290029AE0FF241D
:1018DF0002122B1AE0FE74092FF582E43401F5830E
:1018EF00EEF090029AE014122B2D80D1900297E027
:1018FF001475F007A490029AF0E4900298F0900209
:10190F0098E0FFC39407501A122B22E0FF90029A1F
:10191F00E02402122B1AEFF090029AE004122B2D02
:09192F0080DC900183E02407F044
:01193800228C
:0F329D0030B5FD122B41122753122B4102224E46
:10004600EC4D6011E8497017ED33EC3304600DE4B4
:10005600FCFFFEFD22E933E8330470F80202961233
:10006600026158046009E4CC248150062850090234
:1000760002A028400302029DC0E0EB4A7044B9800A
:1000860006D0E0FB02028CEF4E701CBD8008EBFF31
:10009600EAFEE9FD80EBE98DF0A4FEE5F002012F12
:1000A600E9CDF9EAFEEBFFEF89F0A4FCE5F0CE8995
:1000B600F0A42EFFE435F0CD89F0A42DFEE435F052
:1000C6008067EF4E7005BD80D780C3EF8BF0A4AC80
:1000D600F0EE8BF0A42CFCE435F0F8EF8AF0A42CBB
:1000E600E5F038FCE433CB8DF0A42CFCE5F03BF8CE
:1000F600EE8AF0A42CFCE5F038F8E433CF89F0A4BE
:100106002CFCE5F038CF3400CE89F0A42FFFE5F0C3
:100116003EFEE433C98DF0A42EFEE5F039CD8AF01B
:10012600A42FFFE5F03EFEE43DFD33D0E0FB500793
:100136000BBB000F0202A0EC2CFCEF33FFEE33FEEC
:06014600ED33FD0202781A
:10014C000202A0EC5D046005E859047003020296FB
:10015C00120261580460F6EC4860F2EC7004FDFE8B
:10016C00FF22C860DB2481C85009C3986002500686
:10017C0002029D9850CAF582E9294B4A7005AB8260
:10018C0002028C75F0007C1A7880C3EF9BEE9AED1E
:10019C0099400DC3EF9BFFEE9AFEED99FDE842F0FE
:1001AC00DC23ACF0D0E0FFD0E0FED0E0FDAB822051
:1001BC00E7101BEB60BAEC2CFCEF33FFEE33FEEDDB
:1001CC0033FD020278E803F830E705C0F075F00063
:1001DC00EF2FFFEE33FEED33FD40B830E7C280AABF
:1001EC0075F020800E75F010800575F0087D007E8E
:1001FC00007F003392D530D50312048BEC334010C2
:10020C00EF33FFEE33FEED33FDEC33FCD5F0ED2296
:0E021C00E5F0247EA2D513CC92E7CDCEFF22D2
:10022A00EDD2E7CD33EC3392D524814006E4FFFECC
:10023A00FDFC22FCE4CFCECDCC24E0501174FF802B
:10024A00EDC3CC13CCCD13CDCE13CECF13CF0470C8
:07025A00F030D5DE02048B39
:10026100E9D2E7C933E833F892D5EDD2E7CD33ECE3
:0702710033FC5002B2D5225C
:10027800EC30E7100FBF000C0EBE00080DBD0004E7
:100288000BEB6014A2D5EB13FCED92E7FD2274FF93
:10029800FCFDFEFF22E480F8A2D574FF13FC7D80EC
:0302A800E480EF00
:030000000233596F
:0C335900787FE4F6D8FD75812102317503
:1002AB00BB010689828A83E0225002E722BBFE0251
:0902BB00E32289828A83E4932284
:1002C400BB010CE58229F582E5833AF583E02250EF
:1002D40006E92582F8E622BBFE06E92582F8E22239
:0D02E400E58229F582E5833AF583E4932253
:1002F100EF8DF0A4A8F0CF8CF0A428CE8DF0A42E21
:02030100FE22DA
:10030300BC000BBE0029EF8DF084FFADF022E4CCDE
:10031300F875F008EF2FFFEE33FEEC33FCEE9DECA7
:10032300984005FCEE9DFE0FD5F0E9E4CEFD22EDED
:10033300F8F5F0EE8420D21CFEADF075F008EF2F37
:10034300FFED33FD4007985006D5F0F222C398FD28
:050353000FD5F0EA22C5
:10035800C5F0F8A3E028F0C5F0F8E5821582700230
:060368001583E038F022CD
:10036E00E88FF0A4CC8BF0A42CFCE98EF0A42CFC2E
:10037E008AF0EDA42CFCEA8EF0A4CDA8F08BF0A4AC
:10038E002DCC3825F0FDE98FF0A42CCD35F0FCEB0B
:10039E008EF0A4FEA9F0EB8FF0A4CFC5F02ECD39D0
:0F03AE00FEE43CFCEAA42DCE35F0FDE43CFC223D
:1003BD0075F008758200EF2FFFEE33FECD33CDCCF7
:1003CD0033CCC58233C5829BED9AEC99E58298407A
:1003DD000CF582EE9BFEED9AFDEC99FC0FD5F0D657
:1003ED00E4CEFBE4CDFAE4CCF9A88222B800C1B981
:1003FD000059BA002DEC8BF084CFCECDFCE5F0CBBF
:10040D00F97818EF2FFFEE33FEED33FDEC33FCEBF7
:10041D0033FB10D703994004EB99FB0FD8E5E4F9B2
:10042D00FA227818EF2FFFEE33FEED33FDEC33FC9F
:10043D00C933C910D7059BE99A4007EC9BFCE99A93
:10044D00F90FD8E0E4C9FAE4CCFB2275F010EF2FD8
:10045D00FFEE33FEED33FDCC33CCC833C810D707D8
:10046D009BEC9AE899400AED9BFDEC9AFCE899F813
:0E047D000FD5F0DAE4CDFBE4CCFAE4C8F922A6
:102CC400C2D5E830E70FB2D5E4C39BFBE49AFAE43B
:102CD40099F9E498F8EC30E717B2D5122CFA1203FC
:102CE400F9E4C39BFBE49AFAE499F9E498F88003C5
:102CF4001203F930D50DE4C39FFFE49EFEE49DFD6D
:042D0400E49CFC222D
:0E048B00C3E49FFFE49EFEE49DFDE49CFC2282
:10049900EB9FF5F0EA9E42F0E99D42F0E89C45F0B9
:0104A9002230
:1004AA00E8600FECC313FCED13FDEE13FEEF13FF30
:0304BA00D8F12254
:1004BD00E86010ECA2E713FCED13FDEE13FEEF1355
:0404CD00FFD8F02242
:1004D100E8600FEFC333FFEE33FEED33FDEC33FC89
:0304E100D8F1222D
:0C04E400ECF0A3EDF0A3EEF0A3EFF0228B
:00000001FF
